:1000000026C040C03FC03EC03DC0D3C03BC03AC088
:1000100039C038C037C036C035C034C033C0000026
:10002000000037000000000038000000000036002B
:10003000020202020202020202020102040810206D
:100040002004100801020000040000000000112438
:100050001FBECFE5D1E0DEBFCDBF10E0A0E6B0E02F
:10006000E0EDF7E002C005900D92A636B107D9F792
:1000700010E0A6E6B0E001C01D92A937B107E1F794
:10008000E9D1A4C3BDCF0F931F93CF93DF938C010E
:10009000C0E0D0E0C801E1D0219683E0C83ED80797
:1000A000C9F7DF91CF911F910F910895EF92FF92C1
:1000B0000F931F9382E0F6D09093670080936600C1
:1000C00083E0F0D09093690080936800009166000F
:1000D00010916700809168009091690065E070E080
:1000E0004FD30A9690936C0080936B00E0906B0066
:1000F000F0906C00222717FD2095322FC901B8011E
:1001000048D220EA3AE147EF5FEBCFD220E030E07F
:100110004AEF54E4ACD10FD28B019C01C70168EEC9
:1001200073E040D380E090E0061B170B280B390BDF
:10013000009360001093610020936200309363008D
:1001400080916D0061E00AD180916B0090916C000C
:1001500084D080916D0060E001D180916000909129
:100160006100A0916200B09163008DDF1F910F913B
:10017000FF90EF900895809164002ED1019739F49B
:1001800080916A00882319F010926A008FDF8091B5
:10019000640022D1892B19F481E080936A000895CC
:1001A00080916D0061E09BD08091640060E097D009
:1001B00008951F920F920FB60F9211242F933F9321
:1001C0004F935F936F937F938F939F93AF93BF935F
:1001D0002091730030917400409175005091760029
:1001E00070917700DA01C9010296A11DB11D672F38
:1001F0006A5F6D3730F06D57DA01C9010396A11DB2
:10020000B11D609377008093730090937400A09366
:100210007500B093760080916F0090917000A0916E
:100220007100B09172000196A11DB11D80936F0005
:1002300090937000A0937100B0937200BF91AF9142
:100240009F918F917F916F915F914F913F912F91EE
:100250000F900FBE0F901F901895019739F00197DE
:1002600029F0880F991F01970197F1F70895789465
:100270008AB582608ABD8AB581608ABD83B7826093
:1002800083BF83B7816083BF89B7826089BF80B72E
:10029000826080BF80B7816080BF329A319A309A85
:1002A000379A0895982F863008F09650977080916D
:1002B00078008295880F880F807C892B87B9369AC1
:1002C0003699FECF24B145B1942F80E030E0282B41
:1002D000392BC90108958CB580648CBD0895CF93E6
:1002E000DF93482F50E0CA01865C9F4FFC01349198
:1002F000405D5F4FFA018491882369F190E0880F97
:10030000991FFC01E25EFF4FA591B491FC01EC5DE9
:10031000FF4FC591D491662351F42FB7F8948C9177
:10032000932F909589238C93888189230BC0623009
:1003300061F42FB7F8948C91932F909589238C9327
:100340008881832B88832FBF06C09FB7F8948C9138
:10035000832B8C939FBFDF91CF910895482F50E05E
:10036000CA018C5B9F4FFC012491CA01865C9F4FA0
:10037000FC019491405D5F4FFA013491332359F1B0
:100380002223A9F0223081F0233018F4213079F4AF
:1003900008C0233011F0243051F48CB58F7D8CBD12
:1003A00006C08AB58F7702C08AB58F7D8ABDE32FDC
:1003B000F0E0EE0FFF1FEC5DFF4FA591B4912FB75A
:1003C000F894662321F48C919095892302C08C9136
:1003D000892B8C932FBF0895682F70E0CB018C5B25
:1003E0009F4FFC012491CB01865C9F4FFC014491FF
:1003F000605D7F4FFB019491992319F420E030E078
:1004000027C02223A9F0223081F0233018F42130B4
:1004100079F408C0233011F0243051F48CB58F7D6D
:100420008CBD06C08AB58F7702C08AB58F7D8ABD24
:10043000892F90E0880F991F865D9F4FFC01A59141
:10044000B4918C9120E030E0842311F021E030E081
:10045000C9010895CF93DF930ADF3DDFA1DEC0E03D
:10046000D0E089DE2097E9F3CBDDFBCF5058BB27E6
:10047000AA270ED0E0C0D1D030F0D6D020F031F491
:100480009F3F11F41EF4C6C00EF4E095E7FBBCC01C
:10049000E92FE2D080F3BA17620773078407950744
:1004A00018F071F49EF5FAC00EF4E0950B2EBA2FF9
:1004B000A02D0B01B90190010C01CA01A00111246A
:1004C000FF27591B99F0593F50F4503E68F11A1616
:1004D000F040A22F232F342F4427585FF3CF4695A7
:1004E00037952795A795F0405395C9F77EF41F16C9
:1004F000BA0B620B730B840BBAF09150A1F0FF0F93
:10050000BB1F661F771F881FC2F70EC0BA0F621F7E
:10051000731F841F48F4879577956795B795F7956E
:100520009E3F08F0B3CF9395880F08F09927EE0F00
:1005300097958795089598D088F09F5790F0B92F98
:100540009927B751A0F0D1F0660F771F881F991F28
:100550001AF0BA95C9F712C0B13081F09FD0B1E05E
:1005600008959CC0672F782F8827B85F39F0B93F6E
:10057000CCF3869577956795B395D9F73EF490952A
:100580008095709561957F4F8F4F9F4F0895E894A8
:1005900009C097FB3EF490958095709561957F4FCB
:1005A0008F4F9F4F9923A9F0F92F96E9BB27939579
:1005B000F695879577956795B795F111F8CFFAF489
:1005C000BB0F11F460FF1BC06F5F7F4F8F4F9F4FBA
:1005D00016C0882311F096E911C0772321F09EE818
:1005E000872F762F05C0662371F096E8862F70E07E
:1005F00060E02AF09A95660F771F881FDAF7880F58
:100600009695879597F9089597F99F6780E870E028
:1006100060E008959FEF80EC089500240A94161678
:10062000170618060906089500240A9412161306E0
:10063000140605060895092E0394000C11F488236E
:1006400052F0BB0F40F4BF2B11F460FF04C06F5F8A
:100650007F4F8F4F9F4F089557FD9058440F551F60
:1006600059F05F3F71F04795880F97FB991F61F034
:100670009F3F79F087950895121613061406551FAB
:10068000F2CF4695F1DF08C0161617061806991F17
:10069000F1CF86957105610508940895E894BB270C
:1006A00066277727CB0197F908950AD0C4CFB5DF25
:1006B00028F0BADF18F0952309F0A6CFABCFEFCF23
:1006C000CBDFA8F39923D9F35523C9F3950F50E055
:1006D000551FAA27EE27FF27BB27002408946795FC
:1006E00020F4E20FF31FB41F0A1E220F331F441F12
:1006F000AA1F6695A9F7779530F4F30FB41F0A1E69
:10070000121E08F46395330F441FAA1F221F76950B
:1007100099F7879520F4B40F0A1E121E631F440F29
:10072000AA1F221F331F8695A9F7862F712D602DD2
:1007300011249F5750408AF0E1F088234AF0EE0FD1
:10074000FF1FBB1F661F771F881F91505040A9F7DE
:100750009E3F510570F058CFA2CF5F3FECF3983E1B
:10076000DCF3869577956795B795F795E7959F5F45
:10077000C1F7FE2B880F911D9695879597F90895DF
:100780005527002480FF02C0060E571F660F771FF3
:100790006115710521F096958795009799F7952F2A
:1007A000802D0895AA1BBB1B51E107C0AA1FBB1FC8
:1007B000A617B70710F0A61BB70B881F991F5A95ED
:1007C000A9F780959095BC01CD010895F894FFCFCD
:0607D000D0070000070045
:00000001FF
